:1000000012C02CC02BC02AC029C028C027C026C0BF
:1000100025C024C023C0C1C321C020C01FC01EC032
:100020001DC01CC01BC011241FBECFE5D4E0DEBF25
:10003000CDBF10E0A0E6B0E0E4EFFDE002C0059027
:100040000D92A43FB107D9F721E0A4EFB0E001C0C1
:100050001D92A034B207E1F78ED4CAC6D1CF21B326
:10006000242B21BB32B3242F2095232332B3432BDF
:100070003FB7F894FC01680F791FA2E3B0E0E617E0
:10008000F70719F43FBF78940895819198E0E894B8
:100090004C93000087FF2C93880F07F407F408F4B3
:1000A0002C939A95A9F7EBCF9B01220F331F620F78
:1000B000731FD5DF83E893E00197F1F700C00000DC
:1000C000089540E8F1CF660F771F660F771F40E86D
:1000D000C6DF83E893E00197F1F700C000000895C0
:1000E00040E8BDCF8091F40081111092F400089592
:1000F000282F80911101289FC0011124EFEFF0E01B
:10010000BF0169D4462F80911001289FC00111249E
:10011000BF0161D4362F80911201289FC0011124A4
:10012000BF0159D4862FE5EFF0E04183308382830D
:10013000339691E0E031F907C1F769E070E085EFAF
:1001400090E0BFCFE5EFF0E0818360834283339698
:1001500091E0E031F907C1F769E070E085EF90E0E8
:10016000B0CFCF93DF93C5EFD0E0698183E090E01B
:10017000B0D5688182E090E0ACD56A8181E090E002
:10018000A8D589818C8F88818B8F8A818D8FDF9113
:10019000CF910895CF93DF9300D0CDB7DEB79A8388
:1001A000898389819A8190931401809313016981D5
:1001B0007A8180E090E00F900F90DF91CF9189C518
:1001C000CF92DF92EF92FF920F931F93CF93DF9323
:1001D00000D000D000D01F92CDB7DEB719821A82AE
:1001E0001B821F821E826FE670E00AD58C01CE0151
:1001F00001966C01F12CEE24EA9401151105B9F574
:100200004B816A8189819EDFACDF8E2D71DF8E810B
:100210009F81C0DF88EA90E02ED38091F60090E0C5
:1002200035D38CE224D38091F50090E02FD38CE27B
:100230001ED38091F70090E029D385EA90E01BD38C
:1002400086EB90E018D38E2D90E020D385EA90E0E5
:1002500012D389EC90E00FD38E819F8117D38DE06C
:1002600006D38AE004D381E08093F40006C095E0D1
:10027000F91212C081E790E0FED227960FB6F894EB
:10028000DEBF0FBECDBFDF91CF911F910F91FF90C9
:10029000EF90DF90CF900895E2E0EF15A8F04AE0EC
:1002A00050E0BE016C5F7F4FC801BCD3F601608394
:1002B0008C819D818017910701F5F6018081811164
:1002C0001CC080E990E0D8CFF3E0FF1209C04AE0FB
:1002D00050E0BE016C5F7F4FC801A4D3E62EE8CF8B
:1002E00084E0F812E5CF4AE050E0BE016C5F7F4F3A
:1002F000C80198D37F836E83DBCFF3946FE670E001
:1003000090E080E07DD48C01FFEFCF1ADF0A75CF3B
:10031000CF93DF93E199FECF80E090E0D2D490E0DC
:100320009093140180931301C5EFD0E083E090E037
:10033000C8D4898382E090E0C4D4888381E090E0CF
:10034000C0D48A83239681E0C031D80779F78091A1
:10035000F600809311016091F500609310014091C7
:10036000F70040931201EEDE809113019091140189
:1003700011DF8CED90E07FD28091F60090E086D284
:1003800080EF90E078D28091F50090E07FD280EF0E
:1003900090E071D28091F70090E078D280EF90E009
:1003A0006AD2809113019091140170D285EA90E095
:1003B000DF91CF9160C2CF93C8EC94DE811130C041
:1003C0008C2F96DE8FE59AEE0197F1F700C00000C2
:1003D000C15098F7C2E386DE811122C08FE295E713
:1003E0000197F1F700C00000C150A9F77BDE811131
:1003F00017C08C2F7DDE8FE59AEE0197F1F700C0D4
:100400000000CF5FC93C91F7C4E66CDE811108C0E3
:100410008FE295E70197F1F700C00000C150A9F7FE
:10042000CF910895CF9388EC63DEC5E05BDE811148
:1004300032C08FE295E70197F1F700C00000C1508C
:10044000A9F7C8EC4FDE811126C08C2F51DE87EB57
:100450009BE00197F1F700C00000C15098F788ECCD
:1004600047DEC8EC3FDE811116C08C2F41DE87E0ED
:1004700092E50197F1F700C00000C15098F7CEE176
:1004800031DE811108C087EC9FEA0197F1F700C0C7
:100490000000C150A9F7CF9108952F923F924F923B
:1004A0005F926F927F928F929F92AF92BF92CF9204
:1004B000DF92EF92FF920F931F93CF93DF9300D0C1
:1004C0001F92CDB7DEB78091170190E0FC01EE0FCF
:1004D000FF1FE80FF91FE05AFF4F20812983318069
:1004E0002280019665E070E08AD280931701FC01BA
:1004F000EE0FFF1FE80FF91FE05AFF4F8080821AAE
:10050000990861806318770842804218550810E006
:1005100000E0F12CE12CD12CC12C85E690E09B83EE
:100520008A8344E6A42EB12CDDDD811135C0C801DB
:10053000B50151D2422D460FC701B5014CD2232D32
:10054000260FC601B50147D2862F622F9981890FE8
:10055000F9DD8FE59AEE0197F1F700C000008A817E
:100560009B8101979B838A83C80CD91CE60CF71CDE
:10057000040D151D892BC1F692E39983B3DD81111A
:100580000BC08FE295E70197F1F700C00000998159
:10059000915099839111F2CF0F900F900F90DF91AE
:1005A000CF911F910F91FF90EF90DF90CF90BF9070
:1005B000AF909F908F907F906F905F904F903F9003
:1005C0002F9008951F93CF93DF93E82F862F6BE230
:1005D000F6D1282F892F880F890F382F330FCFEFAF
:1005E000D0E0AE01431B51091FEF149FC001159FBE
:1005F000900D1124BE01EFD1F62F462F319FC0017F
:100600001124BE01E8D1962F223019F140F42223A3
:1006100021F0213061F02F2F90E04FEF0AC02330FE
:10062000E1F02430C1F7462F2FEF90E002C020E028
:100630009FEF6E2F70E0FB01EE0FFF1FE60FF71F1D
:10064000EB50FF4F418390832283DF91CF911F9125
:100650000895262F9FEF40E0ECCF9F2F2FEFFBCF89
:10066000CF93DF93D0E0C0E0609116016D0F8C2F27
:10067000A9DFCF5FD45EC930B9F769E070E085EFDC
:1006800090E01FDD809116018E5F80931601C3E01C
:1006900029DD811108C08FE295E70197F1F700C0CD
:1006A0000000C150A9F7DF91CF910895CF93DF9358
:1006B00080911501823051F138F4882399F181300D
:1006C00059F1109215011FC0833089F0CFEFD0E0AF
:1006D0008430B9F707DD811116C0C2DF8FE295E7DC
:1006E0000197F1F700C000002197A1F705C0D5DE02
:1006F000D4DED3DED2DED1DE809115018F5F85306E
:1007000000F780931501DF91CF9108958BDE8ADE8B
:1007100089DE88DE87DEF0CF4EDE4DDE4CDE4BDE3E
:100720004ADEEACF409112016091100180911101DF
:1007300009DD8FEFDDDCC4EFD1E0D4DC8111E3CF44
:100740008FE295E70197F1F700C000002197A9F724
:10075000D3CF8FE295E70197F1F700C0000008952D
:100760002FEF8EE994E2215080409040E1F700C0E5
:10077000000072D080EE90E05AD08F9AC9DD789454
:10078000089587B38C6287BB709A8DB180658DB9EF
:1007900008958FB9779BFECF08951F920F920FB6E1
:1007A0000F9211242F933F934F935F936F937F93F7
:1007B0008F939F93AF93BF93EF93FF938CB19091DF
:1007C00019019F3110F010921901E091190191E087
:1007D0009E0F90931901F0E0E25EFE4F808384301B
:1007E00021F08D3011F08A3089F4E0911901F0E0A8
:1007F000E25EFE4F108210921901E0911A01F09111
:100800001B01309719F08EE191E00995FF91EF916E
:10081000BF91AF919F918F917F916F915F914F9118
:100820003F912F910F900FBE0F901F9018959093AE
:100830001B0180931A010895E0911A01F0911B01A8
:10084000309749F080911801882329F08EE191E0DA
:1008500009951092180108958898899A8AB1886933
:100860008AB986EA80BD10BC8DE489B908955D9B84
:10087000FECF8CB90895CF93DF93EC01899181115C
:1008800003C0DF91CF910895F2DFF8CFCF93DF93CC
:1008900000D000D000D01F92CDB7DEB74AE0BE0135
:1008A0006F5F7F4FD8D1CE010196E5DF27960FB657
:1008B000F894DEBF0FBECDBFDF91CF910895DF92D8
:1008C000EF92FF920F931F93CF93DF93CDB7DEB7D5
:1008D000C05CD1090FB6F894DEBF0FBECDBFFE01DC
:1008E000319690ECDF011D929A95E9F77F01DF01C7
:1008F000362F50EC27E090E074E016E0D12E9830CF
:1009000081F1903189F1983189F1032F10E0022EA5
:1009100002C0159507950A94E2F700FF2AC0DC9201
:100920009F5F2150515011965111E9CFF8948F01DA
:1009300000541F4FF70181917F012BDF0E151F051A
:10094000C9F77894C054DF4F0FB6F894DEBF0FBEDE
:10095000CDBFDF91CF911F910F91FF90EF90DF906E
:100960000895382F27E0D1CF342FFCCF362F90E0D9
:10097000CCCF7C93D5CFF4DE8091130190911401FC
:1009800082309105B1F030F4009761F00197A1F742
:1009900012DDF2CF8430910581F068F0059761F7A0
:1009A00085DEEACF8FE295E70197F1F700C00000FE
:1009B000E3CF38DDE1CF71DDDFCF52DEDDCF991B34
:1009C00079E004C0991F961708F0961B881F7A9546
:1009D000C9F780950895AA1BBB1B51E107C0AA1F48
:1009E000BB1FA617B70710F0A61BB70B881F991FD0
:1009F0005A95A9F780959095BC01CD01089597FB74
:100A0000072E16F4009406D077FD08D0E4DF07FC2B
:100A100005D03EF4909581959F4F0895709561950E
:100A20007F4F0895B0E0A0E0E7E1F5E09FC15C01F1
:100A30006B017A016115710519F0FB0191838083C7
:100A4000E114F10449F0C7010297839728F060E0B0
:100A500070E0CB019AC05E01E5012196F50110819D
:100A6000812F90E0C5D0892BB1F71D3209F055C018
:100A70002196F501118101E0E114F10409F4ABC004
:100A8000F0E1EF16F10409F08CC0103341F48881D5
:100A90008F7D883509F081C0198122960260E0E1DE
:100AA000EE2EF12C88248A94982CA82CFFE0BF2EDF
:100AB00020E060E070E0CB0127010F2C000C6608FD
:100AC0007708FE0150ED352E310E39E0331538F43C
:100AD0003FEB310F3A3198F549EC342E310E3E148C
:100AE0001F04B4F52F3FB1F086169706A806B90685
:100AF00068F1A3019201FED0232D30E050E040E0E8
:100B0000620F731F841F951F621773078407950771
:100B1000E8F021E021961081D4CF1B3221F4E501C9
:100B20002296F501118100E0A7CF78E0E72EF12CA5
:100B300088248A94982CA82C6FE1B62EB9CF3FE96F
:100B4000310F3A3128F439EA332EC8CF2FEFE2CFF4
:100B5000C114D10431F02223E1F02197F601D183B1
:100B6000C08300FF07C090958095709561957F4F79
:100B70008F4F9F4F2F3F49F482E290E090933F01C7
:100B800080933E016FEF7FEFCB01CDB7DEB7E1E1A0
:100B900009C101FFE6CF2297E1CF10E3E114F10490
:100BA00021F23AE0E316F104E1F080E1E816F10405
:100BB00009F475CFE8E0EE16F10409F4B9CF6FEF50
:100BC0007FEFCB0197010F2C000C440B550BA1D0EC
:100BD00049015A016DCF103309F459CF9AE0E92E3B
:100BE000F12C89E9882E982CA82C89E1B82E60CFA9
:100BF000911154C0803219F089508550D0F7089572
:100C00004CE151E001D00895FA01A191B081009723
:100C100019F41097E1F0CD01DC01CD010D90002019
:100C200011F4C00113C0FB012191222319F02015FA
:100C3000D9F7F3CFFB012191201519F41E921196DB
:100C400006C02223C1F70D900020A1F7D001FA01C0
:100C5000A193B0830895BB274A3031F4992322F43D
:100C6000BDE2909581959F4F01C0BB27FB015527A1
:100C7000AA27880F991FAA1FA41710F0A41B8395F9
:100C80005051B9F7A05DAA3308F0A95DA193009770
:100C900079F7B111B1931192CB0103C0992788273D
:100CA0000895DC01FC01672F71917723E1F73297FA
:100CB00004C07C916D9370836291AE17BF07C8F337
:100CC0000895E199FECF9FBB8EBBE09A99278DB323
:100CD0000895262FE199FECF9FBB8EBBE09A019726
:100CE0000DB2021631F02DBB0FB6F894E29AE19ADC
:100CF0000FBE0895DB018F939F932DD0BF91AF91CD
:100D0000A29F800D911DA39F900DB29F900D112465
:100D10000895A1E21A2EAA1BBB1BFD010DC0AA1F3C
:100D2000BB1FEE1FFF1FA217B307E407F50720F054
:100D3000A21BB30BE40BF50B661F771F881F991FCF
:100D40001A9469F760957095809590959B01AC0118
:100D5000BD01CF01089540D0A59F900DB49F900D87
:100D6000A49F800D911D112408952F923F924F92C0
:100D70005F926F927F928F929F92AF92BF92CF922B
:100D8000DF92EF92FF920F931F93CF93DF93CDB734
:100D9000DEB7CA1BDB0B0FB6F894DEBF0FBECDBFAC
:100DA00009942A88398848885F846E847D848C847D
:100DB0009B84AA84B984C884DF80EE80FD800C8186
:100DC0001B81AA81B981CE0FD11D0FB6F894DEBF69
:100DD0000FBECDBFED010895A29FB001B39FC0012A
:100DE000A39F01D0B29F700D811D1124911D089504
:040DF000F894FFCFA5
:100DF400FF000000FF000000FFFFFF0000FFFF2CCA
:100E040000496E76616C6964206E756D626572204E
:100E14006F6620617267756D656E74732E0D0A00BE
:100E24004572726F72206E756D62657220706172A8
:100E340073696E672E0D0A003E204E657720636F3E
:100E44006C6F723A20003E204E65772062726967AB
:100E540068746E6573733A20003E204E6577206394
:100E64006F6C6F72206D6F64653A20003E2053658D
:100E74007474696E6773206C6F616465643A2000F2
:040E84002C2000001E
:00000001FF
